:020000040000FA
:040000000000F82CD8
:06000A00831603138113AD
:100010000F308600831203138601193083160313F1
:1000200099001815181283120313981783160313D7
:100030009816831203173F08AA3A03192128482467
:100040001928EE3085244824831203173F08EE3A1E
:10005000031D2E28203083120313860083120317FA
:10006000AD0183120317AE01482483120317AE1F9C
:100070006628831203173F08F03A031D42288312B3
:100080000317AD17831203173F08773A031D34286F
:100090008030831203172D0583120317A000200858
:1000A0000319342883120317AE1383120317200891
:1000B00083120317AD0083120313861E6128860185
:1000C000A42B2030831203138600A42BFF3083124D
:1000D0000317AF00831203173F08113A0319B02822
:1000E0003F08123A0319B9283F08143A0319B428F3
:1000F0003F081F3A0319C7283F08273A0319CC289D
:100100003F08583A0319D6283F08593A0319C2281C
:100110003F08773A0319D1283F087C3A0319E028B1
:100120003F087E3A0319DB283F08843A0319F52873
:100130003F08E03A0319A8283F08E13A0319AC2820
:100140003F08F03A031D022983120317AD17342824
:10015000831203172D17342883120317AE17342880
:1001600083120317AF010229023083120317AF0075
:100170000229831203172D1BA42B053083120317AA
:10018000AF000229043083120317AF0002290C309C
:1001900083120317AF0002290D3083120317AF003B
:1001A00002291A3083120317AF0002291B30831271
:1001B0000317AF000229193083120317AF00022979
:1001C000831203172E1C0229831203172D1F0229E5
:1001D000AD1BA42B83120313861EF0288601A42BCB
:1001E0002030831203138600A42B83120317AD1F44
:1001F000FE282030831203138600A42B83120313DE
:100200008601A42B831203172F08FF3A03198629AE
:1002100007302F0583120317A0000130A10020082A
:10022000003C0319192983120317A10D013E031C79
:10023000132983120317AF1D6B292F1E5829831210
:100240000317AD1BA42B8312031721088312031776
:10025000AE06831203172F08193A031D4029831293
:100260000317AE1C3A29831203130C1E33291230D4
:1002700099004029831203130C1E3A29103099006B
:10028000ED3085240E30831203172E0583120317D9
:10029000AF000310AF0C2F088524482483120317E6
:1002A0003F08FA3A0319A42B831203138601A42BE7
:1002B00083120317AD1F6429831203172109A000BD
:1002C00083120317AE05A42B831203172108831290
:1002D0000317AE04A42B831203172D1F73290310D9
:1002E00083120317A10D83120317AD1F7F298312F9
:1002F00003172109A00083120317AD05A42B831255
:100300000317210883120317AD04A42B83120317CC
:10031000AD1BA42B831203172E1DB5297330FF00CC
:100320006930282483120317A00083120317AF003B
:1003300073308312031720020318B52997308312F4
:100340000317AF072F08F03E83120317A0000530F4
:100350000318013EA1002008FE002108FF008030A4
:100360008C2583120317AF009A2B1A30FF00003040
:10037000282483120317A00083120317AF001A303A
:100380008312031720020318F82961308312031720
:10039000AF07831203172D080F390319E5298312BC
:1003A0000317AF12831203172D080C390319DB2929
:1003B000831203172F13831203172D080339031910
:1003C0009A2B83120317AF179A2B831203172D084A
:1003D00030390319EF29203083120317AF06831237
:1003E0000317AE1D9A2B203083120317AF069A2BEA
:1003F0000230FE002A30FF001A30FA23831203175E
:10040000A00083120317AF002A30831203172002C3
:100410000318232A83120317AF0A2F088316031326
:100420009B001C141A0883120317AF0083160313D2
:100430001A080A3A031D9A2B831203130C1E1C2A56
:100440000D3099009A2B0330FE006930FF002A30EE
:10045000FA2383120317A00083120317AF00693039
:1004600083120317200203185F2A83120317AF0AAF
:10047000831203172D0830390319412A83120317F9
:10048000AF0A831203172F08831603139B001C1453
:100490001A0883120317AF00831203172D080C39B3
:1004A0000319552A831203172F13831203172D08DC
:1004B000033903199A2B83120317AF179A2B7D3038
:1004C000FF007730282483120317A000831203173C
:1004D000AF007D308312031720020318912A893060
:1004E00083120317AF07831203130C1E732A1B30EA
:1004F0009900831203130C1E792A5B309900831232
:1005000003130C1E7F2A3130831203172F07831227
:1005100003139900831203130C1E8A2A7E3099005C
:10052000A42B7730FF007330282483120317A00018
:1005300083120317AF0077308312031720020318CA
:10054000BD2A8D3083120317AF07831203130C1ECD
:10055000A52A1B309900831203130C1EAB2A5B30B3
:100560009900831203130C1EB12A41308312031722
:100570002F07831203139900A42BC7238312031799
:10058000A00083120317AF0030308312031720023C
:100590000318592B831203130C1ECA2A1B3099000F
:1005A000831203130C1ED02A5B30990083120317A9
:1005B000AF0A2F08C03E83120317A00005300318AE
:1005C000013EA1002008FE002108FF0080308C259C
:1005D00083120317A20022080319062B83120313A8
:1005E0000C1EEE2A831203172F08C03E8312031736
:1005F000A00005300318013EA1002008FE002108DC
:10060000FF0080308C258312031399008312031797
:10061000AF0A2F08C03E83120317A000053003184D
:10062000013EA1002008FE002108FF0080308C253B
:1006300083120317A20022080319362B8312031317
:100640000C1E1E2B831203172F08C03E83120317A4
:10065000A00005300318013EA1002008FE0021087B
:10066000FF0080308C258312031399008312031737
:10067000AF0A2F08C03E83120317A00005300318ED
:10068000013EA1002008FE002108FF0080308C25DB
:1006900083120317A20022080319A42B8312031349
:1006A0000C1E4E2B8312031722088312031399008A
:1006B000A42B831203130C1E592B21309900831293
:1006C00003130C1E5F2B831203173F0E0F39831287
:1006D0000317A000F03EA00005300318013EA10062
:1006E0002008FE002108FF0080308C2583120313B0
:1006F0009900831203130C1E792B0F3083120317FA
:100700003F0583120317A000F03EA0000530031838
:10071000013EA1002008FE002108FF0080308C254A
:10072000831203139900831203130C1E932B2030A2
:100730009900A42B831203130C1E9A2B8312031708
:100740002F0883120313990083120317AD1FB42BD4
:10075000831203173F08123A031DB42B83120317A9
:100760002E1CB42B2E10C12B831203172D1FC12B4F
:10077000831203173F08123A031DC12B831203177C
:100780002E143F3083120317AD053428080083125E
:100790000317A90130308312031729020318F62B1F
:1007A0002908C03EAA0005300318013EAB002A0804
:1007B000FE002B08FF0080308C2583120317AC004D
:1007C000831203173F060319F62B831203172C0815
:1007D000831203173F020318F12B303083120317E3
:1007E000A900043083120317A907CA2B8312031729
:1007F0002908080083120317A6007F08A7007E08B7
:10080000A80083120317270826020318242C2608A1
:10081000831603139B001C14831203173F088316CF
:1008200003131A060319242C1A08831203173F0214
:1008300003181F2C831203172708A600012C83120C
:1008400003172808A607012C83120317260808009F
:1008500083120317A4007F08A5008312031725083D
:1008600024020318442C2408831603139B001C1431
:10087000831203173F08831603131A060319442C27
:1008800083120317A40A2D2C8312031724080800CF
:100890000F308316031386008312031306184C2CA3
:1008A00083120313061C502C83120317B201083065
:1008B0008312031732020318722C031083120317DA
:1008C000BF0C831203130618612C861D6A2C831239
:1008D0000317BF1783120313061C6A2C8312031716
:1008E000B20A572C831203130618722C83120313B7
:1008F000061C762C8312031306187A2C861D842C72
:1009000083120313061C802C080083120317A30014
:1009100083120317B0010E308316031386000F30C5
:1009200083120317B10083120317B1033108031DAB
:10093000932C073083160313860083120317B1012B
:1009400008308312031731020318C62C83120313D5
:100950000618A62C83120317231CB62C8312031728
:10096000B00A0F30831603138600BA2C07308316A3
:1009700003138600031083120317A30C83120313BF
:10098000061CBE2C83120317B10AA02C831203137A
:100990000618C62C83120317301CD32C073083167D
:1009A00003138600D72C0F3083160313860083129F
:1009B0000313061CD72C831203130618DB2C0F30ED
:1009C00083160313860083120313061CE32C831281
:1009D00003138619E72C831203130618EB2C8312DA
:1009E0000313861DEF2C83120313061CF32C08003F
:1009F0000030FE000630FF008030000000009F2520
:100A00000000000083120317B4007F08B300023017
:100A1000B5000630B600831203173308B700340858
:100A2000B800FF30B307031CB403370838040319B8
:100A3000882D04303507B700B801B80D3608B8075F
:100A40003708FE003808FF008030000000009F25B6
:100A50000000000083120317BA007F08B9003508B0
:100A6000FE003608FF008030000000009F250000D7
:100A7000000083120317BC00B8007F08BB00B7005A
:100A800002303507B700B801B80D3608B807370887
:100A9000FE003808FF008030000000009F250000A5
:100AA000000083120317B800BE007F08B700BD0026
:100AB000831203173908BD003A08BE00FF30B9079A
:100AC000031CBA033D083E040319812D3B08FE00B8
:100AD0003C08FF008030000000008C250000000072
:100AE00083120317BD003708840083133818831757
:100AF0003D088000BB0A0319BC0AB70A0319B80AEB
:100B0000582D063083120317B5070318B60A0B2DAC
:100B10000000000005280800003A0319932D803AD0
:100B200003199A2D00347E08840083137F188317DD
:100B3000000808007F088A007E0882000800003A4A
:100B40000319A72D803A0319B12DFF0100347E0847
:100B5000840083137F1883170008FF00840A0008AD
:100B60000800000000009A25FD00FE0FFF03FF0AA9
:100B7000000000009A25FC007D08FF007C080800AA
:100B80000134323430347E3403345B344534003441
:100B900004345B344334003405345B344134003472
:100BA00006345B34423400340734323434347E3417
:100BB0000934323431347E340A34313439347E34B9
:100BC0000B34313437347E340C345B3444340034E9
:100BD0007834323433347E348334313438347E34B0
:100BE00030343134323433343434353436343734C9
:100BF000383439344134423443344434453446344F
:100C0000023400340E3406343F34013401340034ED
:100C10000F340634403401340134003400340034DD
:02400E00713F00
:104200001C3432342134233424342B3434343334C6
:1042100043343B3442344B343A34313444344D34F7
:1042200015342D341B342C343C342A341D342234C0
:1042300035341A340D340934293420345A340A34CC
:104240006634083476341B3479342B347B342D3483
:104250007C342A340E3460347E34163431342134C4
:104260001E34323440342534343424342634333448
:1042700023342E3435342534363436345E343D34EC
:10428000373426343E3438342A3441342C343C34E8
:1042900045343034293446343934283449342E34C2
:1042A0003E344A342F343F344C343B343A344E3469
:1042B0002D345F3452342734223454345B347B340D
:1042C00055343D342B345B345D347D345D345C34A3
:1042D0007C347034693472347A346B3473347434AB
:1042E0006C3475347D347534723474346B346C349E
:0A42F0007034713469347D347A347F
:00000001FF
